:020000040000FA
:0C0000000000000000EF02F017EF02F01B
:080018005CEF02F09EA8FED788
:10002000AD6E1200096A086EFF0E0826092200D084
:10003000D8A01200030E076EE60E02D8F5D7076AA5
:10004000FE0F066EE86A075AD8A0120000000606E6
:1000500000D0F8D71750135C1C6E11E21C6C1350C3
:1000600017C013F0176E145018C014F0186E155006
:1000700019C015F0196E16501AC016F01A6E1A0E25
:100080001C6074D0175272E01B6A14501F6E18184F
:100090001E6E148E188E080E1C5E08E31AC01BF02C
:1000A00019C01AF018C019F0186AF5D71C2607E015
:1000B000D890183219321A321B321C2EF9D71EAEC4
:1000C00033D01A50165E1950155A1850145A07E2B8
:1000D000D880000E165615561456800E1F1A1B6C2B
:1000E00004E01606000E155A145A040E1C6E14660F
:1000F0000DD015C014F016C015F01BC016F01B6A09
:10010000080E135E29E31C2EF2D726D014BE08D0A9
:10011000D8901B36163615361436132EF7D71CD04A
:100120001BAE22D01B6A0FD01A501626195015226A
:100130001850142206E31432153216321B32134AB9
:100140000DD01BAE11D0163E0FD0153E0DD0143E73
:100150000BD0D8801690EFD7136A02D01D82136897
:10016000166A156A800E146E1FAE149E1650120089
:100170001450126E18181E6E175051E0135252E0B0
:10018000135E7F0E03E2132603E24BD013264CE2EC
:1001900016C010F015C011F0128E188E180E1F6EBA
:1001A000166A156A146A0BD01A50105C195011584F
:1001B00011E3116E126A1A50105E0BD004E218504F
:1001C000125CF2E007E31A50105E1950115A1850F1
:1001D000125AD880163615361436103611361236A5
:1001E0001F2EECD714BE07D013521BE01E3213068D
:1001F0001F2A1E36E3D707E21A50105E1950115A13
:100200001850125A17E3163E15D0153E13D0143E5F
:1002100011D0143215321632133E0CD005D01D8683
:1002200004D01D84136A02D01D821368166A156AF1
:10023000800E146E1EAE149E165012001450126ED4
:1002400018181E6E1350D8A417503AE013267E0ECD
:1002500003E3135E03E336D0135E31E316C010F000
:1002600015C011F0128E188E166A156A146A180ECF
:100270001F6E12321132103206E31A501626195030
:100280001522185014221432153216321F2EF1D7AF
:1002900014BE07D0163615361436135210E0130666
:1002A000123416E3163E14D0153E12D0143E10D070
:1002B000D880143215321632133E0AD003D01D8472
:1002C000136A02D01D821368166A156A800E146EB6
:1002D0001EAE149E1650120013C01FF0145016C00C
:1002E00014F0166E16361F3216321D6A16361F3679
:1002F00002E31D841D7E06E11D801F6A166A156AD1
:10030000146A0BD01F2803E0D880163206D0D8908C
:10031000163202E11D8201D01D861DB604D01DA239
:100320000FD01DB407D07F0E166EFF0E156E146E23
:10033000136E23D0800E166E01D0166A000EF6D70B
:100340001DB0FBD7136A9F0E1F60EBD77E0E1F6494
:10035000F4D79E0E1F5C07E0D89016321532143287
:1003600013321F2AF6D71DA408D0D880000E1356CA
:1003700014561556165616AEE0D713501200136ECB
:10038000146A156A166A1E9E0AD01E9E16AE07D003
:10039000D880000E13561456155616561E8E960EFD
:1003A0001F6E165209E0080E1F2614C013F015C068
:1003B00014F016C015F011D015520FE1080E1F5E93
:1003C000145007E1080E1F5E135002E1165010D0C2
:1003D000136A156E13C014F0136A15BE06D0D890B8
:1003E0001336143615361F06F8D71EAE159E1F504D
:1003F00013C016F0136E155014C015F0146E1200D1
:10040000400E1D6E006A4F0EAF6EB06A240EAC6EC9
:10041000900EAB6E00010F0EC16E070EB46EC69A41
:10042000470E926EE00E936EC00E946E59D09EAA47
:1004300017D0ABA404D0AE50AE50AB881100ABA225
:1004400005D0AE50AE50AB98AB881100352A00EE07
:1004500037F03550E926000EEA22AECFEFFF11004B
:10046000F2A409D0F294224A232AD6CF20F0D7CF83
:1004700021F0817A11003550365C0AE0362A00EE10
:1004800037F03650E926000EEA22EF50346E01D0E4
:1004900034681200376A356A366A9D8A9F8AF28EFE
:1004A000F28C12009D9A376A356A366AAE50AE50A9
:1004B000AB98AB889D8A1200F29EE0CF40F3D8CF74
:1004C00041F3E8CF42F3F28E0001A192F29E40C3C5
:1004D000E0FF41C3D8FF42C3E8FFF28E10001000D6
:1004E000CB68BE6A0C0EBD6E9494BB6ABA6E9492D1
:1004F000050ECA6E7F0ECB6EBE6A0C0EBD6E949456
:10050000BB6ABA6E9492939A8A9ACF0EBD16000E69
:10051000BD12000EBE6ECF0EBA16000EBA12000E3D
:10052000BB6E2F6A939A8A8A320E12EC00F0939A6D
:100530008A9AB0DFB7DFCD6AF294F28A870ED56E61
:10054000B16AA192A082D08EA292B00EB16E3DD9B6
:10055000030137692D500EEC00F0420E0EEC00F056
:10056000400E0EEC00F00001D6CF20F0D7CF21F0E6
:1005700082DF34C024F0BC0E245C07E3FE0E245C52
:1005800002E3F9D002D0266AF6D024AE21D0266A42
:100590008B0E245C05E124C026F02768286817D05C
:1005A0009B0E245C05E124C026F029682A680FD040
:1005B000AB0E245C05E124C026F02B682C6807D024
:1005C000BB0E245C04E124C026F02D682E68D3D035
:1005D000265202E1D0D0CFD08B0E265C1DE1272819
:1005E00003E124C027F016D024C028F04B0E275C6E
:1005F00007E1CF0EBA16000EBA12000EBB6E09D07C
:100600004C0E275C06E1CF0EBD16000EBD12000E8B
:10061000BE6E2768B0D0AFD09B0E265CD8A45AD04F
:10062000292803E124C029F053D024C02AF02A52FB
:1006300015E14B0E295C07E1CF0EBA16000EBA1277
:10064000000EBB6E09D04C0E295C06E1CF0EBD1624
:10065000000EBD12000EBE6E29688DD02FA037D0BF
:100660004B0E295C19E101EE37F0D8902A34E926C7
:10067000000EEA22EECF02F0EFCF03F000EE02F020
:10068000CF0EBA16EE38300BBA12ED30F36EEF30F3
:10069000BB6EF332BB321BD04C0E295C18E102EE6C
:1006A00037F0D8902A34E926000EEA22EECF02F085
:1006B000EFCF03F000EE02F0CF0EBD16EE38300B98
:1006C000BD12ED30F36EEF30BE6EF332BE322968EC
:1006D00052D051D0AB0E265CD8A441D02B2803E1D8
:1006E00024C02BF03AD024C02CF04B0E2B5C19E127
:1006F00001EE37F0D8902C34E926000EEA22EECF36
:1007000002F0EFCF03F000EE02F0CF0EBA16EE3893
:10071000300BBA12ED30F36EEF30BB6EF332BB32FA
:100720001BD04C0E2B5C18E102EE37F0D8902C3425
:10073000E926000EEA22EECF02F0EFCF03F000EE42
:1007400002F0CF0EBD16EE38300BBD12ED30F36E59
:10075000EF30BE6EF332BE322B680DD00CD0BB0E24
:10076000265C09E12D2803E124C02DF003D024C02C
:100770002EF003D800D08170F6D6420E2D5C14E125
:100780002E520FE12F90CF0EBA16000EBA12000EA5
:10079000BB6ECF0EBD16000EBD12000EBE6E2F6AD0
:1007A00002D02F802F680FD07B0E2D5C0CE1CF0E76
:1007B000BA16000EBA12000EBB6ECF0EBD16000E9A
:1007C000BD12000EBE6E2D6812000101386B376B32
:1007D0003A6BD20E396F010E0201366FA60E356FDD
:1007E00035C302F036C303F039C204F03AC205F053
:1007F0000450025C136E05500358146EC1EC01F0F6
:1008000016C03FF315C03EF314C03DF313C03CF3D4
:100810001A6A196A7E0E186E850E176E3FC316F09F
:100820003EC315F03DC314F03CC313F0B8EC00F028
:1008300016C03FF315C03EF314C03DF313C03CF3A4
:10084000020E256E00017F0E255CD8B049D039C15B
:1008500002F03AC103F02550BFEC01F03FC31AF09B
:100860003EC319F03DC318F03CC317F01EEC01F075
:1008700016C00FF015C00EF014C00DF013C00CF030
:1008800002C013F003C014F0C1EC01F00FC01AF065
:100890000EC019F00DC018F00CC017F02AEC00F0D3
:1008A00016C03BF315C03AF314C039F313C038F344
:1008B0003BC316F03AC315F039C314F038C313F034
:1008C0006CEC01F001EE37F0D8902534E926000EEB
:1008D000EA2213C0EEFF14C0EFFF252AD8A0B2D73A
:1008E0000201386B376B3A6B630E396F010E0301EF
:1008F000366F6A0E356F35C302F036C303F039C266
:1009000004F03AC205F00450025C136E055003581F
:10091000146EC1EC01F016C03FF315C03EF314C0D5
:100920003DF313C03CF31A6A196A7E0E186E850EE9
:10093000176E3FC316F03EC315F03DC314F03CC321
:1009400013F0B8EC00F016C03FF315C03EF314C02E
:100950003DF313C03CF3020E256E00017F0E255CB3
:10096000D8B049D039C202F03AC203F02550BFECEA
:1009700001F03FC31AF03EC319F03DC318F03CC369
:1009800017F01EEC01F016C00FF015C00EF014C0E9
:100990000DF013C00CF002C013F003C014F0C1EC52
:1009A00001F00FC01AF00EC019F00DC018F00CC005
:1009B00017F02AEC00F016C03BF315C03AF314C050
:1009C00039F313C038F33BC316F03AC315F039C3FB
:1009D00014F038C313F06CEC01F002EE37F0D8904D
:1009E0002534E926000EEA2213C0EEFF14C0EFFF03
:0A09F000252AD8A0B2D71200FFD7C5
:020000040030CA
:0300010006170ED1
:020005008580F4
:060008000FC00FE00F40E5
:00000001FF
